:020000020000FC
:100000009CCE1895189518951895189518951895CB
:1000100018951895189518951895189518951118FC
:1000200028E008F4100E00FC101A159407941FB76E
:100030002A95B9F70895112428E0069408F4100EC3
:10004000179407941FB72A95C9F708950F931F9324
:100050002F933F93AF93BF93B0E0A2EB19912991F7
:10006000399100E215C00F931F932F933F93AF93E5
:10007000BF93B0E0A2EB19912991399100E237FFCB
:1000800007C00DE21095209530951E0D2D1D3D1DCC
:100090000F9300E20D9300E310582649384910F001
:1000A0000395FACF6894003311F400E2E8940D93BD
:1000B00010582946374600E3105422443F4010F0C0
:1000C0000395FACF2EF06894003311F400E2E8941F
:1000D0000D93105C2D4B304F00E3105A26483140F1
:1000E00010F00395FACF2EF06894003311F400E27B
:1000F000E8940D93105629473E4F00E310512742D4
:10010000304010F00395FACF2EF06894003311F4CC
:1001100000E2E8940D93105F284D3F4F00E3185E16
:10012000234010F00395FBCF2EF06894003311F4B8
:1001300000E2E8940D9318512C4F00E31456204030
:1001400010F00395FBCF2EF06894003311F400E219
:10015000E8940D931C5900E31A5010F00395FCCF5E
:100160001EF0003309F400E20D93165C1D9310E0BD
:100170001D93E894A2EBB0E00D910032E9F31297E1
:100180000F910C93BF91AF913F912F911F910F91C0
:1001900008956F9266240F931F932F93E894152E62
:1001A000012E112717FC139507FC139510FD689479
:1001B000012D35DF127811FD02C00EF411601FBF52
:1001C0002F911F910F91200111244F93089447956F
:1001D00002C0469529F008F4100E17940794F9CF41
:1001E0000F930FB700780FBF17FC08940F914F9132
:1001F00010010F931F932F93152E002E012DE894BD
:1002000007FD689407FD019516DF13782EF410940E
:10021000009401E0000E121E17FC11601FBF2F9109
:100220001F910F915608300C411C561C0F931F93C1
:100230002F93112E042E012DE89407FD689407FDDD
:100240000195F9DE13782EF41094009401E0000E6D
:10025000121E17FC11601FBF2F911F910F9156089E
:10026000300C411C561C6F900895AF92AA241124A3
:100270004F930894479502C0469529F008F4100E54
:1002800017940794F9CF0F930FB700780FBF17FC9F
:1002900008940F914F9110010F931F932F93E8949F
:1002A000162E012E112717FC139507FC139510FD30
:1002B0006894012DB4DE127811FD02C00EF41160B5
:1002C0001FBF2F911F910F91502C612C442411249A
:1002D0005F930894579502C0569529F008F4100EC4
:1002E00017940794F9CF0F930FB700780FBF17FC3F
:1002F00008940F915F91300C411C0F931F932F9323
:10030000162E002E012DE89407FD689407FD019537
:1003100092DE13782EF41094009401E0000E121E69
:1003200017FC11601FBF2F911F910F916A08400C9D
:10033000511C6A1C0F931F932F93112E042E012D15
:10034000E89407FD689407FD019575DE13782EF497
:100350001094009401E0000E121E17FC11601FBFE4
:100360002F911F910F915A086A08300C411C5A1C9A
:100370006A1C0F931F932F93112E052E012DE894C5
:1003800007FD689407FD019556DE13782EF410944E
:10039000009401E0000E121E17FC11601FBF2F9188
:1003A0001F910F916A08400C511C6A1CAF90089570
:1003B0008F929F92AF92AA2411244F93089447954D
:1003C00002C0469529F008F4100E17940794F9CF4F
:1003D0000F930FB700780FBF17FC08940F914F9140
:1003E000100111245F930894579502C0569529F087
:1003F00008F4110E17940794F9CF0F930FB70078F4
:100400000FBF17FC08940F915F9120010F931F936A
:100410002F93E894162E012E112717FC139507FC35
:10042000139510FD6894012DFADD127811FD02C0BC
:100430000EF411601FBF2F911F910F9130010F9388
:100440001F932F93162E012E012DE89407FD68941B
:1004500007FD0195F0DD13782EF41094009401E06F
:10046000000E121E17FC11601FBF2F911F910F91DC
:100470007A08400111245F930894579502C056955D
:1004800029F008F4100E17940794F9CF0F930FB7C3
:1004900000780FBF17FC08940F915F91300C411C3E
:1004A000581C691C7A1C0F931F932F93122E052E34
:1004B000012DE89407FD689407FD0195BCDD1378D4
:1004C0002EF41094009401E0000E121E17FC11602F
:1004D0001FBF2F911F910F917A08400111244F9354
:1004E0000894479502C0469529F008F4110E179418
:1004F0000794F9CF0F930FB700780FBF17FC08943C
:100500000F914F91300C411C581C691C7A1C0F93A1
:100510001F932F93162E002E012DE89407FD68944B
:1005200007FD019588DD13782EF41094009401E006
:10053000000E121E17FC11601FBF2F911F910F910B
:100540006A087A08401C511C6A1C7A1C0F931F937E
:100550002F93122E042E012DE89407FD689407FDB9
:10056000019569DD13782EF41094009401E0000EDB
:10057000121E17FC11601FBF2F911F910F916A0867
:100580007A08401C511C6A1C7A1CAF909F908F9077
:100590000895AF92AA246624552444240F931F93F0
:1005A0002F93102E042E012DE89407FD689407FD6B
:1005B000019541DD13782EF41094009401E0000EB3
:1005C000121E17FC11601FBF2F911F910F91100178
:1005D0000F931F932F93102E052E012DE89407FDE6
:1005E000689407FD019527DD13782EF4109400948C
:1005F00001E0000E121E17FC11601FBF2F911F910A
:100600000F915A086A08300C411C5A1C6A1C0F933F
:100610001F932F93102E062E012DE89407FD68944A
:1006200007FD019508DD13782EF41094009401E085
:10063000000E121E17FC11601FBF2F911F910F910A
:100640006A08400C511C6A1C0F931F932F93E89467
:10065000102E072E112717FC139507FC139510FD7C
:100660006894012DDCDC127811FD02C00EF41160DB
:100670001FBF2F911F910F91500C611CAF900895D7
:100680008F929F92AF92AA2411244F93089447957A
:1006900002C0469529F008F4100E17940794F9CF7C
:1006A0000F930FB700780FBF17FC08940F914F916D
:1006B000100111246F930894679502C0669529F084
:1006C00008F4100E17940794F9CF0F930FB7007822
:1006D0000FBF17FC08940F916F9120010F931F9388
:1006E0002F93E894172E012E112717FC139507FC62
:1006F000139510FD6894012D92DC127811FD02C053
:100700000EF411601FBF2F911F910F9130010F93B5
:100710001F932F93172E002E012DE89407FD689448
:1007200007FD019588DC13782EF41094009401E005
:10073000000E121E17FC11601FBF2F911F910F9109
:1007400040017A0811245F930894579502C056958A
:1007500029F008F4100E17940794F9CF0F930FB7F0
:1007600000780FBF17FC08940F915F91300C411C6B
:10077000581C691C7A1C0F931F932F93112E042E63
:10078000012DE89407FD689407FD019554DC13786A
:100790002EF41094009401E0000E121E17FC11605C
:1007A0001FBF2F911F910F915A086A087A08300CC9
:1007B000411C5A1C6A1C7A1C0F931F932F93112EF5
:1007C000052E012DE89407FD689407FD019533DCA3
:1007D00013782EF41094009401E0000E121E17FC02
:1007E00011601FBF2F911F910F916A087A08400C6A
:1007F000511C6A1C7A1C0F931F932F93112E062EE7
:10080000012DE89407FD689407FD019514DC137829
:100810002EF41094009401E0000E121E17FC1160DB
:100820001FBF2F911F910F917A08500C611C7A1CE9
:10083000AF909F908F900895AF92BF92CF92DF922A
:10084000EF92EE2411244F930894479502C04695E9
:1008500029F008F4100E17940794F9CF0F930FB7EF
:1008600000780FBF17FC08940F914F9110011124CD
:100870005F930894579502C0569529F008F4110E1D
:1008800017940794F9CF0F930FB700780FBF17FC99
:1008900008940F915F91200111246F93089467953C
:1008A00002C0669529F008F4120E17940794F9CF48
:1008B0000F930FB700780FBF17FC08940F916F913B
:1008C00030010F931F932F93E894172E032E1127B7
:1008D00017FC139507FC139510FD6894012D9FDB01
:1008E000127811FD02C00EF411601FBF2F911F91ED
:1008F0000F9140010F931F932F93172E022E012D5E
:10090000E89407FD689407FD019595DB13782EF4B4
:100910001094009401E0000E121E17FC11601FBF1E
:100920002F911F910F9160019E0811246F930894DD
:10093000679502C0669529F008F4110E1794079484
:10094000F9CF0F930FB700780FBF17FC08940F91E2
:100950006F91500111245F930894579502C05695EA
:1009600029F008F4100E17940794F9CF0F930FB7DE
:1009700000780FBF17FC08940F915F91300C411C59
:100980005A1C6B1C7C1C8D1C9E1C0F931F932F9359
:10099000132E062E012DE89407FD689407FD01959E
:1009A0004ADB13782EF41094009401E0000E121E1E
:1009B00017FC11601FBF2F911F910F9160019E08BE
:1009C00011245F930894579502C0569529F008F4B6
:1009D000120E17940794F9CF0F930FB700780FBF3B
:1009E00017FC08940F915F91500111244F930894C4
:1009F000479502C0469529F008F4110E1794079404
:100A0000F9CF0F930FB700780FBF17FC08940F9121
:100A10004F91300C411C5A1C6B1C7C1C8D1C9E1C65
:100A20000F931F932F93172E012E012DE89407FD8E
:100A3000689407FD0195FFDA13782EF41094009462
:100A400001E0000E121E17FC11601FBF2F911F91B5
:100A50000F9150019E088E0811244F9308944795DA
:100A600002C0469529F008F4120E17940794F9CFA6
:100A70000F930FB700780FBF17FC08940F914F9199
:100A8000400C511C6A1C7B1C8E1C9E1C0F931F93D8
:100A90002F93132E052E012DE89407FD689407FD72
:100AA0000195C9DA13782EF41094009401E0000E39
:100AB000121E17FC11601FBF2F911F910F91500143
:100AC0009E088E0811246F930894679502C066955E
:100AD00029F008F4100E17940794F9CF0F930FB76D
:100AE00000780FBF17FC08940F916F91400C511CB8
:100AF0006A1C7B1C8E1C9E1C0F931F932F93132E1E
:100B0000042E012DE89407FD689407FD019593DA02
:100B100013782EF41094009401E0000E121E17FCBE
:100B200011601FBF2F911F910F919E088E087E08A4
:100B3000500C611C7E1C8E1C9E1C0F931F932F93C8
:100B4000172E002E012DE89407FD689407FD0195EE
:100B500072DA13782EF41094009401E0000E121E45
:100B600017FC11601FBF2F911F910F919E088E08D7
:100B70007E08500C611C7E1C8E1C9E1CEF90DF902A
:100B8000CF90BF90AF900895AF92AA24442411242F
:100B90004F930894479502C0469529F008F4100E2B
:100BA00017940794F9CF0F930FB700780FBF17FC76
:100BB00008940F914F9110010F931F932F93172EAD
:100BC000002E012DE89407FD689407FD019533DAA6
:100BD00013782EF41094009401E0000E121E17FCFE
:100BE00011601FBF2F911F910F91502C612C112468
:100BF0005F930894579502C0569529F008F4100E9B
:100C000017940794F9CF0F930FB700780FBF17FC15
:100C100008940F915F91300C411C5A1C6A1C1124DE
:100C20006F930894679502C0669529F008F4100E3A
:100C300017940794F9CF0F930FB700780FBF17FCE5
:100C400008940F916F91400C511C6A1CAF9008954D
:100C50008F929F92AF92AA2411244F9308944795A4
:100C600002C0469529F008F4100E17940794F9CFA6
:100C70000F930FB700780FBF17FC08940F914F9197
:100C8000100111246F930894679502C0669529F0AE
:100C900008F4100E17940794F9CF0F930FB700784C
:100CA0000FBF17FC08940F916F9120010F931F93B2
:100CB0002F93172E012E012DE89407FD689407FD50
:100CC0000195B9D913782EF41094009401E0000E28
:100CD000121E17FC11601FBF2F911F910F91300141
:100CE0000F931F932F93172E002E012DE89407FDCD
:100CF000689407FD01959FD913782EF41094009401
:100D000001E0000E121E17FC11601FBF2F911F91F2
:100D10000F9140017A0811245F930894579502C0FF
:100D2000569529F008F4100E17940794F9CF0F93F5
:100D30000FB700780FBF17FC08940F915F91300C2C
:100D4000411C581C691C7A1C11241F930894179588
:100D500002C0169529F008F4140E17940794F9CFE1
:100D60000F930FB700780FBF17FC08940F911F91D6
:100D7000300C411C5A1C6A1C7A1C11241F930894C5
:100D8000179502C0169529F008F4150E17940794CC
:100D9000F9CF0F930FB700780FBF17FC08940F918E
:100DA0001F91400C511C6A1C7A1C11241F9308943B
:100DB000179502C0169529F008F4160E179407949B
:100DC000F9CF0F930FB700780FBF17FC08940F915E
:100DD0001F91500C611C7A1CAF909F908F900895CA
:100DE000D0E0C6EC09931993299339934993599309
:100DF000699379938993202E312E422E532E569447
:100E0000479437942794420D531D641D751DD0E0FF
:100E1000C6EC09931993299339934993599369938C
:100E200079938993222433244424552480E2440F67
:100E3000551F661F771F221C331C441C551C20168F
:100E400031064206530628F0201A310A420A530A94
:100E500043958A9561F7022D132D242D352DD0E071
:100E6000C6EC89917991699159914991399129916A
:100E70001991099108950027C098C198B898B99818
:100E80000895B89A06D5000000000000B89801D572
:100E9000000000000000689401C0E8940C2D00F9E7
:100EA000B99AF7D4F6D40894001F01C0000F69F076
:100EB000B89A18F40000B99802C0B99A00C0E9D4F1
:100EC000B898B09BFECFE5D4F1CFB89AB998E1D4E9
:100ED000000000000000B898B09BFECF0000B19960
:100EE00035C0D7D4000000000000089511E0B89A82
:100EF000B998CFD4000000000000B898B09BFECF96
:100F00008894B1990894C5D40000111F80F7B89A4D
:100F10000FB706FF03C00000B99803C0B99A0000DC
:100F20000000B7D4B898B09BFECFB3D40895B89A58
:100F3000B99AAFD4000000000000B898AAD400000D
:100F400000000000B998A5D400000895A2D4C19A69
:100F5000EEDFB898B9980895212EA5DF92DF2E1400
:100F600011F406D001C008D019932A94C1F708954E
:100F70006894BCDFDCDF0895E894B8DF089517D0EB
:100F800000918100003609F0089506E7000FC02E99
:100F900084DF02EF88DF05E086DF05EF84DF08E409
:100FA00082DF04EF80DF0AE67EDFC1DF089506E717
:100FB000000FC02E72DF00ED76DF63DFD9DF109304
:100FC0008100089506E7000FC02E67DF18E1D0E02A
:100FD000C0E608E8C1DF06E7000FC02E5EDF11E0C3
:100FE000D0E0C8E701EAB8DF06E7000FC02E55DF02
:100FF00017E0D0E0C9E701EEAFDF00917F0000937A
:10100000800000917C0010917D00202F312F3F70D7
:101010002295422F207F232B4F7043FD406F20935A
:101020007C0040937D0000917E00202F312F32956F
:101030003F702295207F232B02950F7003FD006FD8
:1010400020937E0000937F00089506E7000FC02ED6
:1010500024DF04EF28DF0AE626DF69DF06E7000F5A
:10106000C02E1BDF03EF1FDF0CDF82DF197011239F
:10107000A9F713DF18E0D0E0C2E807EF6DDFD0E09A
:10108000C2E809911991299122951295312F2F705B
:10109000107F122B0295202F3F70007F032B2F70A3
:1010A00023971993099329930991199129912295CD
:1010B0001295312F2F70107F122B0295202F3F7029
:1010C000007F032B2F70239719930993299309917C
:1010D0001991229719930993089500918500109111
:1010E00086002091870025951795079525951795DA
:1010F0000795259517950795D0E0CEE909931993A3
:1011000029932595179507954091600050916100AE
:10111000041B150B6627440F551F661FD0E0C6EA57
:10112000499359936993402F512F33D8559447943D
:1011300037945594479437945594479437945594DD
:1011400047943794432D542D652D009164001091E0
:1011500065008BD8772467FC7094330C441C551CB5
:10116000661C771C330C441C551C661C771CD0E095
:10117000C2EA499259926992799240919E005091A7
:101180009F006091A00077270091A6001091A70012
:101190002091A800332727FD3FEF401B510B620B26
:1011A000730B00916200109163002D2D3D2D00D92D
:1011B00075946794579447943794759467945794AB
:1011C0004794379475946794579447943794D0E034
:1011D000CEE93992499259926992D0E0C2EA0991D6
:1011E000199129913991030D141D251D361DD0E04B
:1011F000CAE80993199329933993A801B90105E025
:10120000C8D900E8200E3D1C4D1C5D1C6D1CD0E0B3
:10121000CEE83992499259926992D0E0CAE8499150
:101220005991699179917595679557954795405072
:101230005A4F60407040D0E0CEE94993599369938A
:1012400079937595679557954795759567955795D2
:1012500047958A019B01F0DA7594679457944794F7
:10126000379475946794579447943794759467941A
:10127000579447943794D0E0CEEA399249925992E4
:101280006992D0E0C0E709911991432D542D652D45
:10129000762DF6D9D0E0C2EA299239924992599234
:1012A000D0E0CEE94991599169917991D0E0CEE6AB
:1012B00009911991E5D9220C331C441C551C661C5C
:1012C000D0E0C2EA4991599169917991420D531D3B
:1012D000641D751DD0E0C2EA4993599369937993CF
:1012E0007595679557954795759567955795479562
:1012F000D0E0CCE6099119914D0D5D1D601F711F65
:10130000D0E0C2EA4993599369937993D0E0CEEA49
:101310004991599169917991759567955795479537
:101320007595679557954795D0E0CAE6099119914B
:10133000A7D9659457944794379427946594579404
:1013400047943794279465945794479437942794F7
:10135000D0E0C6EA2992399249925992D0E0C8E683
:1013600009911991D0E0CEE949915991699179910A
:1013700087D965945794479437942794D0E0C6EA68
:101380000991199129913991200E311E421E531E47
:10139000662457FC6094762C759467945794479410
:1013A0007594679457944794D0E0CEE94992599246
:1013B0006992799240E050E860E070E0440D551D7C
:1013C000661D771DD0E0C6E60991199141DC330C0A
:1013D000441C551C661C771CD0E0CEE949925992FA
:1013E000699279927D146D045D044D0409F40895A9
:1013F000D0E0C2E8099119912991332727FD3FEFE9
:1014000040E050E060E17727401B510B620B730B0B
:10141000D0E0C2EA3991099119912991332727FD2A
:101420003FEF35952795179507953595279517958E
:101430000795359527951795079535952795179510
:101440000795401B510B620B730B05E31CE018D989
:10145000D0E0CAE9299239924992599240E050E08D
:1014600060E070E8D0E0CEE90991199129913991B5
:101470002416350646065706A101B20130F4440F82
:10148000551F661F771FACDC05C0AADC220C331C7D
:10149000441C551CD0E0CAE92992399249925992CC
:1014A00055944794379427945594479437942794A8
:1014B0005594479437942794A101B2018101920178
:1014C000BBD9662457FC6094762C330C441C551C05
:1014D000661C771C330C441C551C661C771C330C93
:1014E000441C551C661C771CD0E0C6E70991199175
:1014F000A201B301C5D855944794379455944794A5
:101500003794559447943794559447943794772754
:1015100057FC7FEFD0E0CEE9399249925992799306
:10152000D0E0CAE94991599169917991759567958A
:10153000579547957595679557954795D0E0C4E7BA
:10154000099119919DD8330C441C551C661C771CBD
:10155000330C441C551C661C771C330C441C551C56
:10156000661C771CD0E0C2EA49925992699279923E
:10157000D0E0CEE94991599169917991440D551D79
:10158000661D771DD0E0C2E709911991400F511FE8
:101590006D1D7D1D75956795579547957595679553
:1015A000579547957595679557954795759567959F
:1015B00057954795D0E0CAE9099119912991399138
:1015C000400F511F621F731F405E5C4F6F4F7F4F74
:1015D000D0E0C2E949935993699379930895D0E093
:1015E000CAE8499159916991799140505C426140B2
:1015F0007040D0E0CEE94993599369937993D0E054
:10160000CEE94991599169917991D0E0CEE709915C
:10161000199136D8D0E0CCE7399119912227159548
:1016200037952795159537952795159537952795CE
:10163000159537952795D0E0C8E8699179914427A9
:1016400055277595679557957595679557954D19D4
:101650005D09620B730B4219530964097509405007
:10166000504C6F4F7F4F442777FD4FEF642E550F3F
:10167000661F771F441FD0E0C2EA699379934993AC
:101680006992D0E0CEE94991599169917991D0E080
:10169000CBE7099179DA6594579447943794659428
:1016A000579447943794659457944794379400E03F
:1016B00010E8300E411E5D1C6D1CD0E0C6EA399268
:1016C000499259926992D0E0CEE949915991699134
:1016D0007991D0E0C0E809915CD76594579447941C
:1016E00037946594579447943794432D542D652D22
:1016F000762DD0E0C6EA09911991299139919CD8AB
:1017000095948794779467945794479437949594D5
:10171000879477946794579447943794432D542D26
:10172000652D762D40505040604E7F4FD0E0C9E788
:1017300009911991A5D781019201A3010050104E82
:101740002F4F3F4F4F4F5F4F110F221F331F441F2B
:10175000551F110F221F331F441F551F89019A0166
:10176000D0E0C2EA499159916991799165D8D0E068
:10177000CEE92992399249925992330C441C551C56
:10178000661C771CA201B3018201930155D8220C7B
:10179000331C441C551C661C432D542D652D762D81
:1017A000D0E0C8E70991F0D96594579447943794ED
:1017B0002794659457944794379427946594579445
:1017C0004794379427946594579447943794279473
:1017D000D0E0CEE949915991699179914219530923
:1017E00064097509D0E0CEE94993599369937993D7
:1017F0004D155D056D057D051CF444275527BA017F
:1018000000E010E020E039E140175107620773075C
:1018100014F0A801B9017595679557957595679569
:1018200057957595679557957595679557950027C1
:1018300077FD0FEF452F562F672F702F08EE13E01F
:101840001FD7659457944794379465945794479459
:101850003794D0E0C6E93992499259926992089535
:1018600007D00197E9F7089514D00197E9F7089593
:10187000BF93AF93B7E0A0ED1197F1F7AF91BF9190
:101880000895F6DF0A95E9F7089503D00A95E9F778
:101890000895C895C895089590E084E1E1DF0CE3D0
:1018A000000FC02EFADA00E0FEDA0EEAFCDA03EEF0
:1018B000FADA00E2F8DA00E0F6DA00EBF4DA08EC43
:1018C000F2DA00E0F0DA00E1EEDA01E2ECDA00E070
:1018D000EADA0FE7E8DA02E2E6DA00E0E4DA07E063
:1018E000E2DA00E4E0DA04EADEDA01EADCDA06EA67
:1018F000DADA01E8D8DA0FEFD6DA08EAD4DA0FE359
:10190000D2DA03EDD0DA00E0CEDA05EDCCDA00EF82
:10191000CADA09EDC8DA02E2C6DA0AEDC4DA02E18F
:10192000C2DA0BEDC0DA00E2BEDA0DE8BCDA04E19F
:10193000BADA0FEAB8DAFBDA08950CE3000FC02E2A
:101940001127002713D0A9DA00E4ADDA20E8002738
:10195000AADA2A95E1F7EBDA1395183091F7E7DA6E
:1019600001D008950027112701D00895180195DAB4
:1019700000E099DA1770106B012F95DA01E293DA23
:10198000022D0F7018E011240F930894079502C0E0
:10199000069529F008F4110E17940794F9CF0F93C8
:1019A0000FB700780FBF17FC08940F910F91002D0F
:1019B0007ADA0FE778DA00E476DAB9DA81010895A5
:1019C0002CE3220FC22ED2DF2991222311F010D056
:1019D000FBCFADDAC7DF08952CE3220FC22EC6DF9E
:1019E0002591222311F004D0FBCFA1DABBDF0895AB
:1019F000CF01205238E011242F930894279502C07C
:101A0000269529F008F4130E17940794F9CF0F9335
:101A10000FB700780FBF17FC08940F912F91FAE1D0
:101A2000EAE3E00DF11D39DA00E43DDA05913BDA35
:101A30003A95E1F77CDAFC0108950000000000000F
:101A4000000000065F5F06000000000707000707B0
:101A50000000147F7F147F7F1400242E6B6B3A12DA
:101A60000000476537187C567300307A4F5D377A2F
:101A700048000000060F090F0600001C3E634100ED
:101A800000000041633E1C000000082A3E1C1C3E72
:101A90002A0808083E3E0808000000A0E060000098
:101AA0000000080808080808000000006060000046
:101AB00000006030180C060301003E7F594D7F3E48
:101AC000000042427F7F40400000627359496F66C8
:101AD0000000226349497F360000181C16137F7FDF
:101AE0001000276745457D3900003C7E4B49793021
:101AF0000000036371190F070000367F49497F36E4
:101B00000000064F49693F1E000000006C6C000099
:101B1000000000A0EC6C00000000081C36634100CF
:101B200000001414141414140000004163361C083F
:101B30000000020351590F0600003E7F415D5D1F0A
:101B40001E007C7E13137E7C0000417F7F49497F0D
:101B500036001C3E634141632200417F7F41637F29
:101B60001C00417F7F495D416300417F7F491D012A
:101B700003001C3E6341517372007F7F08087F7F22
:101B8000000000417F7F41000000307040417F3FF6
:101B90000100417F7F081C776300417F7F414060E7
:101BA00070007F7F060C067F7F007F7F060C187F0A
:101BB0007F001C3E6341633E1C00417F7F49090F4B
:101BC00006001E3F21717F5E0000417F7F19396F43
:101BD000460026674D597B32000003417F7F410359
:101BE00000007F7F40407F7F00001F3F60603F1FFD
:101BF00000007F7F3018307F7F0063771C081C77E0
:101C00006300074F78784F0700006773594D4763AB
:101C10007100007F7F41410000000103060C183075
:101C200060000041417F7F000000080C0603060CA5
:101C3000080080808080808080800000030704008E
:101C40000000207454543C784000413F7F44447C61
:101C50003800387C44446C280000307848493F7F85
:101C60004000387C54545C180000487E7F490302D1
:101C7000000098BCA4A4F87C0400417F7F08047C89
:101C8000780000447D7D4000000040C484FD7D005C
:101C90000000417F7F10386C440000417F7F40008E
:101CA00000007C7C0C180C7C78007C7C04047C7824
:101CB0000000387C44447C38000084FCF8A4243CB8
:101CC0001800183C24A4F8FC8400447C78441C18B8
:101CD0000000485C54547424000000043E7F4424F7
:101CE00000003C7C40403C7C40001C3C60603C1C54
:101CF00000003C7C6030607C3C00446C3810386CE8
:101D000044009CBCA0A0FC7C00004C64745C4C644F
:101D1000000008083E77414100000000007777008E
:101D200000004141773E080800000203010302035E
:101D30000100787C4643467C78000FE50DBF02E049
:101D40000EBFDD2401E0E02EC0E0D2E0F0E0E0E6EE
:101D5000D1922197E9F7BC9AC49A78948CD80FD97C
:101D600031D99ADDEADD0BE011E0FEE1E4E634DE94
:101D70000BE014E0FEE1E8E62FDE0BE017E0FEE109
:101D8000ECE62ADE62D9A9D948DA29DC15D093E03D
:101D900088EE66DDB499C498B49BC49AF3CF0395DA
:101DA000FECFB0E0AAED09910D9309910D93099131
:101DB0000D9309910D930895D0E0CEE8F2DFD0E0C5
:101DC000CAED51D1D092BC000091BA000093BB0083
:101DD0000091B9000093BA000EE20093B90000E050
:101DE00011E0D0E0C2EBECDDD0E0C2E9099119913D
:101DF0002991399108511C4F2F4F3F4FD0E0CAED28
:101E00000993199329933993D0E0CAED2CD1D0923C
:101E1000BC000091BA000093BB000091B900009390
:101E2000BA000EE20093B90000E014E0D0E0C2EB8B
:101E3000C7DDD0E0C6E9B5DFD0E0CAED14D1D0925D
:101E4000BB000091B9000093BA000091B800009364
:101E5000B9000EE20093B80001E017E0D0E0C2EB59
:101E6000AFDD0895274300006850610025724800E7
:00000001FF
